:100000002500FB0C0600FF0C0700A405A305580AF9
:10001000A404A3042200E2013108010800080D082D
:10002000010800080008000800086F087608CA08E0
:10003000A408A108E5087208AD085208D208D10842
:10004000DB08D1089C084D081508080849086E0807
:100050004F08750874083108300842080F0847082F
:10006000720861086D086C0869086308680826084A
:10007000420865086E0873086F086E08A4045E05E0
:10008000A4056607470AA404D509A405410A460544
:10009000A404D509D509D509A405760000000000FF
:1000A000000000000000080C3500A404D50903047A
:1000B000A40536036606F605A404D509D509000093
:1000C0000000A405F502550AA404D509D509A40524
:1000D000160234000008A40443045E064305A40588
:1000E0004307770AA4045E04D509D509A40546048C
:1000F000A404D509D509D5090000000000000000BE
:1001000000000000080CA405380017074604170675
:10011000460503043703A404D509D509D509A40568
:10012000F802850A00004605A404D509D509D509B9
:100130000000000000000000A4050008790010067F
:1001400019053006390550065905700679059006DF
:1001500099051106B90519020700790031069905BC
:100160005106B90571061905910639057905190277
:10017000060000086A006B00680069006C006D00F2
:100180006E006F001F0C30001F0C3100A4047000C3
:1001900071007200730074007500760077001E0411
:1001A0003E04A40572007300000804000C023B002A
:1001B0000D06BB051B0227007B002D069B054D0687
:1001C000BB056D061B058D063B057D0446067D05BA
:1001D0007D075B047D065B051B02260007023B00D2
:1001E0001F0C5B01280069007D04BB067D057D07AF
:1001F00009047D06090506023B009B062905BB068E
:1002000049051B0669053B0689050A0239000B02F0
:100210003A0008028E011F0E2A0009028F011F0EEC
:100220002B000A0252013C000B0253011C013B004F
:100230001B023C001F0C8A0150013C011F0C8B016A
:1002400051011C013B000A02990154014A013B0182
:100250000B029A0155014B013B010A02990156011B
:1002600059013B010B029A0157015A013B011B0244
:1002700043073E055E063F0B000000004A0B3E07A9
:100280004A0B1E07460B46041E04490B00000000E3
:1002900000004D0B000000004D0B050C3C00FC0263
:0602A0004F0B00000008F6
:10040000E2016F0A720A750A780A7B0A7E0A810A7B
:10041000840AE201900A950A9A0A9F0AA40AA90A84
:10042000AE0AB30AE201C10AC70ACD0AD40ADB0A3E
:10043000E30AEB0AEE0AE201FB0A000B050B0A0BCA
:100440000F0B140B190B1E0BE2016C0A8D0ABE0A6E
:10045000F20A230B230B230B230BE201300B380B87
:10046000400B480B500B580B600B680B700B780B54
:10047000E201A00BA00BA00BA00BA90BA90BAF0BCB
:10048000AF0BE201B80BBB0BBE0BC40BC90BD70BF8
:10049000D90BE00BE201870B870B870B870B870BD0
:1004A000880B990BB50BE201660A270B800B810BB9
:1004B000A304BA09A305A3043E0914023A009A034F
:1004C0003C003C031C03030EA305530A1A033C0023
:1004D0003C031C03070E240A070C5A01000A0A02F7
:1004E0003B00860A0B023B00860A0E023B00860A8E
:1004F0000F023B00860A10023B00860A11023B00F5
:10050000860A08023B00860A09023B001F0C5B01B9
:100510003700A3046B09A305260B070C5A01090A2F
:10052000A4041002A4053B00B70AA4041102A40508
:100530003B00B70AA4041202A4053B00B70AA404B6
:100540001302A4053B00B70AA4041402A4053B004F
:10055000B70AA4041502A4053B00B70AA4041602B6
:10056000A4053B00B70AA4041702A4053B001F0C16
:100570005B013700A3046B09A305260B070C5A0186
:10058000120A0C023700A3046B09A305F10A0D023D
:100590003700A3046B09A305F10AA3043E09140262
:1005A0001F0E2E00A305F10AA3043E0914021F0E1C
:1005B0002F00A305F10AA3043E0914021F0E300008
:1005C0009E09A305F10AA3043E0914021F0E31007F
:1005D0009E09A305F10A6C006D00F10AA304BA0993
:1005E000A305260BA3043E0914021F0E3B00070CB3
:1005F0005A01A3051B0A1B02A4043000A405220B08
:100600001B02A4043100A405220B1B02A404320027
:10061000A405220B1B02A4043300A405220B1B0219
:10062000A4043400A405220B1B02A4043500A40575
:10063000220B1B02A4043600A405220B1B02A404F7
:100640003700A405260B1F0C5A012C00E30BBA0639
:100650002D0B1F0C5A012D007F0B0F0C5A012D0A78
:100660001D049A061D051D070C041D060C057F0BB5
:100670001D049A061D051D072C041D062C057F0B65
:100680001D049A061D051D074C041D064C057F0B15
:100690001D049A061D051D076C041D066C057F0BC5
:1006A0001D049A061D051D078C041D068C057F0B75
:1006B0001D049A061D051D070D041D060D057F0B63
:1006C0001D049A061D051D072D041D062D057F0B13
:1006D0001D049A061D051D074D041D064D057F0BC3
:1006E0001D049A061D051D076D041D066D057F0B73
:1006F0001D049A061D051D078D041D068D05E30BBF
:10070000E30B1A033C003C031C03070E4A0AE30BED
:10071000EF0C9A004307980BA40478003E061805D6
:100720001E0638051802A4053700A3046B09A305AB
:10073000E30B1A02A4043800070C5801A405380A78
:10074000A4041E0438061E053E0418063E05A40532
:10075000B40BA4043E0418063E05A405B40BA4047F
:100760001E0418061E05A405E30B070C5A01410AD6
:10077000FC0CE501E30B040CE501E30B050237007B
:10078000A3046B09A305E30B7700A3046B09A3057E
:10079000E30B9302A404A3040B09A40537006B091F
:1007A000B302310C9300A30503067300E30B73003F
:1007B000E30B12023700A3046B097200A305E30BDD
:0807C00092024307B2025B0A3A
:021FFE00D40FFE
:00000001FF
